:020000040000FA
:10000000850186018316073085008601831207303B
:100010009F002F288207013402340334043405344E
:1000200006340734083409340A340B340C340D34E4
:100030000E340F343C346D34393401346334383485
:1000400068343534313471343E341F34303419342B
:1000500078346B3461346534683404344034A3013B
:10006000A501A4012330A5006D207B206820051C7C
:10007000462805193728051C4628051D3B28A30AD4
:10008000213023020318A301682037282416682092
:10009000851848282130A5006D200C302307A200C8
:1000A0005D20A20B5028A4012230A5006D207220F3
:1000B0005D205D205D205D202F28FA30A000C83033
:1000C000A10000000000A10B6128A00B5F28080020
:1000D00023080A2024048600080025080A20240496
:1000E000860008006430A2008517862085138420CE
:1000F000A20B742808006430A2008517882085139D
:100100008420A20B7D2808005030892808308928D7
:100110000430A0003230A10000000000A10B8C28A8
:06012000A00B8A28080074
:02400E00103F61
:00000001FF
